:10000000830100308A0004288301B52B9100921BE4
:10001000102812088A001108910A0319920A820016
:100020008313121883171108910A8400000808002E
:10003000423479342034503461346F346C346F344A
:1000400000344C3427346934723472346934673480
:10005000613474346F3472346534203430342E3467
:040060003134003403
:1006A6008C00831205110C08803E802B83120511E5
:1006B6000130802302305F2B8D0004308E005330D2
:1006C6008F008F0B642B8E0B622B8D0B602B83128E
:1006D600080083120515782B0D0892000C088C0A69
:1006E60003198D0A0620831280230D0892000C0838
:1006F60006200038031908006F2B8E000E0E0F39E6
:10070600831290000608F0391004860085158511BD
:100716000E080F3990000608F0391004860085157A
:1007260085110D308F008F0B962B831208008C00DD
:10073600831205150C0E0F3990000608F0391004C7
:100746008600851585110C080F3990000608F039CA
:1007560010048600851585110D308D008D0BB12B8B
:100766008312080083168101810A03308500D03088
:1007760086008312DA230030532321308C000030A8
:100786008D006C234030532318308C0000308D00D0
:100796006C238612061BD32B8612FA3083125F2334
:1007A600061ACD2B8616FA3083125F23CD2B8312C1
:1007B60005110F305F23033086008515851105303E
:1007C6005F238515851121308C008C0BE82B831255
:1007D6008515851105305F23023086008515851144
:1007E6000D308C008C0BF52B2830831280230830BB
:0A07F60080230F3080230630802B93
:02400E0011009F
:00000001FF
